:100000008A110A1205280000090083160E309F008D
:100010008312831681018312831664308F0083124A
:1000200043309F00831601308500831283168601BA
:100030008312051185118316051185110F30860570
:1000400083126430A0000030A100BD2133302A2289
:1000500033302A2233302A2222302A2228302A2200
:100060000F302A2201302A2201302A22861406115A
:1000700001302A224320861006156430A000A10119
:10008000BD21362842281F1483169F171F130030E6
:100090008312A000022283161E088312AC001E08E1
:1000A000AD002C08A0002D08A100A3013230A12131
:1000B000031D98282C08A0002D08A1001630A200CE
:1000C000A3017F21AE002108AF002E08A6002F0853
:1000D000A7002E08A2002F08A3006921AE00250862
:1000E000AF002C08A6002D08A7000730A200A3012E
:1000F0006921B0002508B1003008A0003108A10036
:100100000A30A200A3017F21B0002108B1002E080F
:100110003007AC002F080318013E3107AD002C0852
:10012000143EAC002D080318013E003EAD00B0287F
:100130001F3083050330A600A7012C08A2002D085C
:10014000A3006921AC002508AD002C08A0002D08F3
:10015000A1000230A200A3017F21AC002108AD0064
:100160001F3083052C08A4002D08A5004322E83089
:10017000A0000330A100BD2101302A222C08A000DC
:100180002D08A1000230A300BC30A121031DDF28EF
:10019000743013227230132265301322733013220D
:1001A0002030132264301322753013227230132250
:1001B000653013226430A000A101BD2162291F30E7
:1001C00083052C08A0002D08A1000230A3005830A0
:1001D000A121031DF82864301322753013227230D8
:1001E0001322653013226430A000A101BD216229D1
:1001F0001F3083052C08A0002D08A1000130A300AA
:10020000F430A121031D17296D3013226930132208
:1002100020301322643013227530132272301322DF
:10022000653013226430A000A101BD2162291F3076
:1002300083052C08A0002D08A1000130A3002C305C
:10024000A121031D3229643013226F30132275302F
:10025000132263301322653013226430A000A10101
:10026000BD2162291F3083052C08A0002D08A100A4
:10027000A3016430A121031D582974301322723068
:10028000132265301322733013222030132264307E
:1002900013226F30132275301322C0302A226330AC
:1002A0001322653013226430A000A101BD21622910
:1002B0001F308305703013227530132272301322E1
:1002C00065301322D030A0000730A100BD21080006
:1002D00068291030A800A101A001A70CA60C031CDE
:1002E00077292208A00723080318230FA107A10CD0
:1002F000A00CA50CA40CA80B6D2924080800103034
:10030000A600A501A401210DA40DA50D2208A4029B
:100310002308031C230FA502031895292208A4070C
:1003200023080318230FA5070310A00DA10DA60B8A
:10033000832920080800A2000530AD29A200023060
:10034000AD29A2000630AD29A2000330AD29A200DC
:100350000430AD29A2000130AD29A80023082102F4
:10036000031DB429220820020430031801300319A8
:1003700002302805031DFF300800A0080319C82912
:10038000CF21A00300000000000000000000BD29F4
:10039000A10803190800CF21A103A003BD290C3037
:1003A000A500A50BD129000000001230A200A20B6D
:1003B000DE29E021E021000000000800E021D7292B
:1003C0000D30A400A40BE229000008000A30A802A6
:1003D000031C0800EB290630A802031C0800EB29C7
:1003E0001030A8020001031C013EA902031C0800F2
:1003F000F9290A30A8020001031C013EA902031CCE
:100400000800F929A00DA00DA00D3830A005C130BD
:1004100020049F001430A800E6211F151F190E2A82
:100420000C131F100800A80085150F30860528083A
:10043000F0398604051500000511A80E0F30860559
:100440002808F03986040515000005116430A8005D
:10045000E6210800A80085110F3086052808F0392C
:100460008604051500000511A80E0F308605280822
:10047000F03986040515000005118830A8001330F6
:10048000A900F0210800A7172730A300103054223C
:100490000330A300E8305422A30164305422A301A6
:1004A0000A30542224085F2AA2002508A10024084B
:1004B000A0007F212008031DA713A71B0800303EC2
:0404C00013220800FB
:02400E00700F31
:00000001FF
